:100000002CC056C01BC154C053C057C051C050C0B3
:100010004FC04EC04DC04CC0CFC04AC049C0000008
:1000200000000000000000000000000023456C9864
:10003000C9FF040714233764A0FFFFFFFFFFFFFF82
:10004000FFFFFFFFFF000000000000000000234052
:100050005F7AB4FFFFFFFFFFFF0011241FBECFE553
:10006000D1E0DEBFCDBF20E0A0E6B0E001C01D9230
:10007000A938B207E1F7E2E6F0E085E5808781E0A4
:1000800083831482128286831182AEE6B0E08EEF03
:1000900015968C9315978DEF17968C938BE082872E
:1000A00088E58387612C712C88248A9486D012C1BC
:1000B000A7CF1BBC19BC18BC0895189525B7277E7F
:1000C00025BF29B7226029BF21E022BF019728F070
:1000D00020E188952150E9F7F9CF089588EE93E063
:1000E000EDCF8CE287B986EC86B9369A3699FECF89
:1000F0008FEF809360000895369A3699FECF95B1C0
:100100008091600089270895811101C0D2CF81506C
:1001100090E0FC01E25EFF4FE491EBBDFC01EE5C80
:10012000FF4FE491E9BDFC01EA5BFF4F849188BD7C
:1001300008950F931F93CF93C82F8B01CC2359F0B1
:1001400085E0E2DFC801BADFB4DFC801B7DFC8016C
:10015000B5DFC150F3CFCF911F910F910895CF9389
:10016000DF93D82F64E170E08AE0E3DF84EF91E071
:10017000A5DF8D2F64E6A2D0CAE06C2F9FD0892F17
:1001800068EC70E0D6DFAADF8D2F6C2F97D0D92FC7
:1001900095D0892F68EC70E0CCDFA0DF68EC70E0D0
:1001A0008D2FC7DF9BDF64E170E08AE0C2DF84EF60
:1001B00091E0DF91CF9182CF18958FEF881210C018
:1001C00083EA87B986EC86B93699FECF369A369996
:1001D000FECF85B1833D18F086E0882E01C0812CCA
:1001E0008FE384BBB99AB89ABC9A81E08ABD83BF79
:1001F0009AB590629ABD9AB590689ABD9FEF9DBDE1
:1002000080BF80E68CBD97B328B3892F90E080959E
:1002100090958B7F822B88BBAB9A8BB780628BBF0C
:100220008AB785608ABF85B7806285BF789459DFB9
:100230008CE291E043DF60DF92DFFACF1124882067
:1002400009F01895F89416B834DFB998B898BC98A6
:1002500030E021E094E086B38870222351F08111D0
:1002600027C086E0881510F021E0F5CF20E099E066
:10027000F2CF332319F0882321F01AC031E0811125
:1002800030E085B7877E806185BF892F887011F443
:1002900040E401C040E6892F8770842B81BD85B77B
:1002A000846885BF8B7F85BF78948895F894D3CF79
:1002B0008FE58DBF81E08EBF1FBE7FDF991B79E088
:1002C00004C0991F961708F0961B881F7A95C9F7E6
:0802D00080950895F894FFCF1A
:00000001FF
